:100000009DC0B7C0CFC0CFC0B4C0B3C0B2C0CCC019
:10001000B0C0AFC0AEC0ADC0ACC0ABC0AAC0A9C07C
:10002000A8C0A7C0A6C0A5C0A4C0A3C0A2C0A1C0AC
:10003000A0C09FC09EC09DC09CC09BC000060C126B
:10004000181E242A30363C42484E545A60666C7260
:10005000787E848A90969CA2A8AEB4BAC0C6CCD250
:10006000D8DEE4EAF0F6FFFFFFFFFFFFFFFFFFFF30
:10007000FFFFFFFFFFFFFFFFFFFFFFFFFFFFFFFF90
:10008000FFFFFFFFFFFFFFFFFFFFFFFFFFFFFFFF80
:10009000FFFFFFFFFFFFFFFFFFFFFFFFFFFFFFFF70
:1000A000FFFFFFFFFFFFFFFFFFFFFFFFFFFFFFFF60
:1000B000FFFFFFFFFFFFFFFFFFFFFFFFFFF9F3ED74
:1000C000E7E1DBD5CFC9C3BDB7B1ABA59F99938D90
:1000D00087817B756F69635D57514B453F39332D80
:1000E00027211B150F090000000000000000000080
:1000F0000000000000000000000000000000000000
:1001000000000000000000000000000000000000EF
:1001100000000000000000000000000000000000DF
:1001200000000000000000000000000000000000CF
:1001300000000000000000000000000011241FBEAD
:10014000CFEFD1E0DEBFCDBF11E0A0E0B1E0EEE146
:10015000F5E002C005900D92A434B107D9F721E073
:10016000A4E4B1E001C01D92A436B207E1F72BD19F
:10017000D4C146CF0F931F9300E010E098010617FB
:1001800017072807390759F0EFE9FFE03197F1F732
:1001900000C000000F5F1F4F2F4F3F4FF0CF1F9148
:1001A0000F910895189518951F920F920FB60F9200
:1001B00011248F939F9381E090E090934501809369
:1001C00044019F918F910F900FBE0F901F90189533
:1001D000FC01EC5DFE4FB081AB2FA09525B72062EE
:1001E00025BF1DBC1CBC729A7A9A109245011092D0
:1001F00044019C01220F331FF901E45FFE4F01907F
:10020000F081E02D40814B2B4083F901E65DFE4FEC
:100210000190F081E02D20812A2320831DBC1CBC8D
:1002200088954CB55DB560914401709145019C0184
:10023000220F331F672B11F4CA0102C08FEF9FEF0B
:100240007A98F901E65DFE4F0190F081E02D408142
:100250004B2B4083F901E45FFE4F0190F081E02DCC
:1002600040814A23408395958795F901EA5BFE4FCB
:1002700020813181821B930B97FF02C080E090E0C8
:100280000895DF92EF92FF920F931F93CF93DF9326
:10029000EC01FC01EE0FFF1FEA5BFE4F11821082A2
:1002A00097DF8FE99FE00197F1F700C0000014E0AD
:1002B000D12E00E010E07E01EE0CFF1CCE0188DFA5
:1002C000080F191F8FE99FE00197F1F700C00000A8
:1002D000DA94A1F7F701EA5BFE4F1595079515959E
:1002E000079511830083DF91CF911F910F91FF90AC
:1002F000EF90DF900895EF92FF920F931F93CF93AB
:10030000DF93109263008FEF97E099BD88BD9BBD8E
:100310008ABD1FBC81E08EBD84E08FB985B7877E22
:1003200085BF8BB780638BBF90E0E92E91E0F92EFB
:1003300004E211E0C0E0D0E0D701ED91FD917D0134
:100340009081D8018D918D01809589238083CE0184
:1003500098DF2196C630D10579F7DF91CF911F91B3
:100360000F91FF90EF9008958093B0008091B100BD
:1003700087FFFCCF0895F8DF80E090E008958A3091
:1003800010F4805D01C0895CEFCFCF93C82F8295B8
:100390008F70F5DF8C2F8F70CF91F1CFCF93C82F57
:1003A000892FF3DF8C2FCF91F0CF8AB38F7A8ABB5E
:1003B000D59A80E48093B20086E391E09093610146
:1003C0008093600108958FEF80937400B89AEDDFF9
:1003D000789491DFF894E2E5F1E0819191918F3F7B
:1003E000910519F014F08FEF90E090E8392F382341
:1003F000292F2695C09A332379F0922F0000000010
:1004000000000000000000000000000000000000EC
:1004100000000000C09808C000000000C098922FA3
:1004200000000000000000000000000000000000CC
:100430000000000000002111D9CF90E8392F3823A7
:10044000292F2695C09A332379F0922F00000000BF
:10045000000000000000000000000000000000009C
:1004600000000000C09808C000000000C098922F53
:10047000000000000000000000000000000000007C
:100480000000000000002111D9CF80E8982F9A7059
:100490008695C09A9923A9F0000000000000000092
:1004A000000000000000000000000000000000004C
:1004B000C0980000000000000000000000000000E4
:1004C000E5CF00000000C098000000000000000020
:1004D000000000000000000000000000000081118A
:1004E000D5CF81E0EE35F80709F077CFC098789442
:1004F000EFE3FCE93197F1F700C0000002E511E0FD
:10050000C0E0D0E0CE0164DEF801819391938F01C9
:0E0510002196C630D105B1F75DCFF894FFCF2C
:10051E006300630063006300620062003200320019
:10052E0032003200400040003B003B003B003B00ED
:10053E00380038000102040804023A003A003A007A
:10054E003A00370037000000000200000000BB0137
:04055E000000000099
:00000001FF
